:030000000219FDE5
:03000B000200AA46
:03002B0002018A45
:03005B0002033964
:030073000203265F
:1000800002030406080C10182030406080040608A3
:100090000C10182030406080A0C00003070F1F0D17
:1000A0000D0403060D0503030202C2AF306308C24C
:1000B0006385798AD2AF32C0D0C0E0206221E525C5
:1000C0006016E473E525F4C3334009758A00D263F2
:1000D000F57901D6F58AD262D0E0D0D0D2AF32C362
:1000E000E526334009758A00D263F57901F0F58A77
:1000F000C262E526F4603030682620720DD0E0D070
:10010000D0C295C294C293D2AF32C295C294C29368
:10011000206F0D20660A7414D5E0FDE57BF4529043
:10012000D0E0D0D0D2AF32758A00D263757900C2E8
:100130008DD262212001C4306805206602D295016B
:10014000C4306805206602D29401C4306805206678
:1001500002D29301C4D29230680A2066077410D587
:10016000E0FDD29501C4D29130680A206607741070
:10017000D5E0FDD29401C4D290D29230680A2066B4
:10018000077410D5E0FDD29301C4C2AFC2AD53E6EF
:10019000EFC0D0C0E0D2D3D2AFE57A6009E5776096
:1001A00005757700412F757701C2CEE52A600720DB
:1001B0007449152A21FB7800790020742EE58030DF
:1001C0007E01F430E70278FF53DACF207E0343DA72
:1001D00020307E0343DA10C2D8C271E580307E0140
:1001E000F430E70279FFC3E89970CB306103752AD8
:1001F00040207403752A40885CD27020740DE52B72
:100200006004152B410B43DA01C2D8207002411E55
:10021000A85C206102C270207402411C882278828E
:10022000B60403852224C3E52594404002D264200D
:10023000CF0AD0E0D0D043E610D2AD32C2CF053ADB
:10024000E57A6009E5786005757800611C757801CC
:100250007802E52A6005307402152AC3E55C940132
:100260004005755F004178756000756900E55F24A1
:1002700001F55F5003755FFF7982B7020D306E1D87
:10028000C3E52294324016854C227982B7030E30A2
:100290006E0BC3E52294324004798E8722C3E52396
:1002A000952260084004152341AC0523D8CA05698E
:1002B000E56970021569D56A63756A017805C3E559
:1002C00069956B4057C3E569956C50087801756A6C
:1002D000030202E0C3E569956D50057801756A0176
:1002E000C3E5629524401E7982B704026111206E35
:1002F00014852462E569046003856B69756A01757C
:10030000233C02031CE5622850057562FF6111F56C
:1003100062E5620470067560FF7569FFD0E0D0D0B9
:1003200043E610D2AD32C2AF53E67F7592FA7593B1
:10033000FFC260759104D2AF32C2AF53E6EFC2ADD7
:10034000C0D0C0E0C0F0D2D3D2AFA8FBA9FCE57A00
:100350006007C3E913F9E813F8C2D830710261AB42
:1003600053DACF207E0343DA10307E0343DA20D203
:1003700071E580307E01F420E702618288278928B8
:10038000A19053DACF207E0343DA20307E0343DA94
:1003900010C2D8C271307402A17C7800E580307E32
:1003A00001F430E702A17C885CA16453DACF207E9F
:1003B0000343DA20307E0343DA10C27120610281E8
:1003C0008453DACF207E0343DA10307E0343DA20F1
:1003D000C2D8D27188578958C3E89555F8E995561F
:1003E000F97B007E087A00C3E8948CE994005005FC
:1003F000755B008176882178A2E6A8216055C3E864
:1004000094C8E994005008E4D2E4FB7A0A8151C30D
:10041000E89468E994015008E4D2E3FB7A0F815133
:10042000C3E894D0E994025008E4D2E2FB7A1E813A
:1004300051C3E894A0E994055008E4D2E1FB7A3C6A
:100440008151C3E89498E994085008E4D2E0FB7A1B
:10045000787E00C3E89559FCE9955AFD30E70AEC2F
:10046000F42401FCEDF43400FD755B00C3EC9AED5F
:0D0470009E5003755B018859895A855755C8
:10047D008558567802A164C3E89527F8E99528F9BF
:10048D00307C02A148307B02A148307A02A1412084
:10049D00750281A7E9FDE8FC81C6E9C313F9E813EC
:1004AD00F8307902A141E9C313F9E813F830780265
:1004BD00A141E9C313FDE813FC20612CC3EC941C8E
:1004CD00ED9402400281DDED701EC3EC94C850180E
:1004DD000529E52970021529C3E529940A5002A1C1
:1004ED007C755C00D270A17CE52960021529740031
:1004FD00207F037896E624FAFEE43400FFC3EC9ED9
:10050D00FCED9FFD500678007900A148C3EC94FFE7
:10051D00ED9400400678FF7900A148EC8572F0A4B7
:10052D00C5F0A2F733F87900400302056478FF792E
:10053D0000020564E9C313F9E813F8307C0EE96095
:10054D000278FFC3E81338F8E43400F9C3E894FFE8
:10055D00E99400400278FF885CD270206102A17C92
:10056D00741FF4552F4BF52FC274EB7002D27475B6
:10057D002A40307403752A0A306102A19020740359
:10058D0053DAFE207403752B20D0F0D0E0D0D0D2FA
:10059D00AD43E6103279010205C079030205C07939
:1005AD000A0205C0791E0205C079640205C079C82A
:1005BD000205C07817E4D5E0FDD8FAD9F6227A14F1
:1005CD007B780205E77A107B8C0205E77A0D7BB408
:1005DD000205E77A0B7BC80205E77902E4D291D5D3
:1005ED00E0FDD294D5E0FDC294D5E0FDC291D5E0F9
:1005FD00FDE920E002D29530E002D293E573D5E01B
:10060D00FDE920E002C29530E002C2937496D5E078
:10061D00FDD9C9EAF8D5E0FDD8FBDBBED29122C3E6
:10062D007C007D0075F00005F0EA33FAEB33FB50EA
:10063D00F6EB13FBEA13FAC3E9FFE8FEE89AF8E9D3
:10064D009BF95004EFF9EEF8B3EC33FCED33FDD527
:10065D00F0DFEDF9ECF822E889F08A20D2D4F8A980
:10066D00F07B0030F70B7BFFF42401F8E9F4340044
:10067D00F9E88520F0A4ADF0F8E98520F0A4AFF0FD
:10068D00FEED2EF974003FFA7C04C3EA13FAE91368
:10069D00F9E813F8DCF48BF030F70AE8F42401F8EC
:1006AD00E9F43400F9E889F0C2D4F8A9F02278828F
:1006BD00B6040302075AC3E55C9419401EE52D5498
:1006CD00067018206E3678057994E7146007780A5D
:1006DD001460027812C3E54198401F306E0985649D
:1006ED00627569FF756A01852224E4F544F545F5C7
:1006FD0046F547F548C26E02075AD26E7994E71453
:10070D007013E523F43333F913F8E9540104F9E8D0
:10071D0054FE02074EE714147014E523F4333333FB
:10072D00F913F8E9540304F9E854FC020756E523DC
:10073D00F433333333F913F8E954070404F9E85467
:10074D00F8C39440F8E99400F98844894522C3E53B
:10075D004113F9E54013F8C3E54498F8E54599F9D7
:10076D00500CC3E89480E994FF4016020792C3E849
:10077D00947FE994005003020792787F7900020775
:10078D0092788079FF8849894A22E5492546F8E51E
:10079D004A3547F9854A20E4300701F43548FA30E7
:1007AD00E709C3EA94F040150207D0C3EA940F504D
:1007BD00030207D078FF79FF7A0F0207D07800790E
:1007CD00007AF0C3E5249561500AC3740195245055
:1007DD000B0207EEE54A20E70E0207EEE54A30E789
:1007ED0006884689478A482278A5E6FAC3E5493343
:1007FD00F8E54A33F9120664E930E70BC3E8948053
:10080D00E994FF40130129C3E8947FE99400500255
:10081D000129787F79000129788079FFE820E71593
:10082D00C3E52398F84009C3E8940140030208503A
:10083D007801020850E8F424012523F8400302084A
:10084D005078FF884B2278A6E6FAA847A9481206E9
:10085D0064E930E70CC3E89401E994FF40160208FF
:0F086D0085C3E894FFE99400500302088578FFE3
:10087C007900020885780179FFE920E715C3E54B7B
:10088C0098F84009C3E8940140030208AC780102CF
:10089C0008ACE8F42401254BF840030208AC78FFBF
:1008AC0088242278FFC26420693D206A12D264C376
:1008BC00E541940A4009C3E52594405002C264798D
:1008CC00A1E76023E541601F74FF8541F084853901
:1008DC00F0306A0375F005A4F8C5F0600278FFC328
:1008EC00E895645002A864886322C3E54094C8E587
:1008FC00419400E5635003142107046002F5632260
:10090C007883E6F520120FAA75E8901205A275E817
:10091C0090E5E820ECFBA8BDA9BE121054756E0042
:10092C00756F00C3740013FD7400606613FC7400D3
:10093C002CFC74003DFDECFAEDFBC3E89AE99B40FE
:10094C0014E56E2400F56EE56F3400F56FEA2CFAB1
:10095C00EB3DFB80E5AE6EAF6FC3E56F13F9E56E53
:10096C0013F8C3E913F9E813F87A03C3E913F9E8A8
:10097C0013F8DAF7AA201A7009756E00756F000269
:10098C00099E1AEA6008EE28FEEF39FFDAF88E6E3F
:10099C008F6F2275E890227883E6FFE5E820ECF76C
:1009AC00A8BDA9BE0570C3E57094084052757000CF
:1009BC00E9FA79A0E76044EA7007E571601B020967
:1009CC00D9C3E895716010E5715006600C140209EA
:1009DC00E50460F90209E5E571F571C39472401BF9
:1009EC007561C0C394044013756180C39404400BBB
:1009FC00756140C39404400375610075BB0622EF1A
:100A0C00C39401601F7400601BC3E894FFE9940356
:100A1C005012C3E8956EE9956F5009E561600C15AD
:100A2C0061020A37E561F460020561A861C3E5243F
:100A3C00985002A824C3E89562400AA862E562F4C3
:100A4C00600385626188258826E570B4070375BB51
:100A5C001022743279A787F0A4C5F0A2F733F8C33B
:100A6C00E895614002A86188228824882588268818
:100A7C0064227540007541F022C2AF75C820A8CC25
:100A8C00A9CDAA3A30CF010A75C824D2AFC3EA1354
:100A9C00FAE913F9E813F8AB3BAC3C883B893CC34F
:100AAC00E89BF8E99C20690A547FF9306702619F42
:100ABC0041FCAD3D8A3DF9EA9D547FFA600478FF14
:100ACC0079FFAE3EAF3F8B3E8C3FA83BA93CC3E8C1
:100ADC009EF8E99FF9C3E54113FBE54013FAE82AB8
:100AEC00F540E93BF54150067540FF7541FF614605
:100AFC00AA40AB41AC40AD417E047F02C3EB9404F1
:100B0C0040021E1FC3EB940840021E1FC3ED13FDD1
:100B1C00EC13FCDEF7C3EA9CFAEB9DFBEF6009C318
:100B2C00E913F9E813F8DFF7EA28FAEB39FB8A4006
:100B3C008B4150067BFF8B408B41C3EB94025002E0
:100B4C00D2673069047F0361717892E6FFC3E537A1
:100B5C00948240110FC3E53794A040010FC3EF946A
:100B6C000640027F057E02E541C4540FF9E541C4FD
:100B7C0054F0F8E540C4540F28F8C3E89EFAE99401
:100B8C0000FB4009C3EA9402EB940050047A02E49F
:100B9C00FB61EBAA40AB41EBC4FEEAC4540F4EFC24
:100BAC00C3EA9CFAEB9400FBC3E813C313F8EA28DE
:100BBC00FAEB3400FB8A408B41C3EB94024002C237
:100BCC00677802EBC4FE7B00EAC4540F4EFAC3EA0A
:100BDC0098FA4005C3940250027A027892E6FF30EC
:100BEC00600261EB855192855293D26043E680C3DB
:100BFC00E49AF8E49BF9C3E833F8E933F930670277
:100C0C00817EE8FAE9FBD3E913FDE813FC885189EE
:100C1C0052C3EF94036038EF20E00DE82CF8E93D67
:100C2C00F9ECFAEDFB020C47E828F8E939F9C3E8CE
:100C3C002402F8E93400F97AFE7BFFC3EF940340F9
:100C4C000E8A538B54884D894E8C4F8D5081B288AF
:100C5C005389548A4D8B4E8C4F8D5030691275537D
:0D0C6C00F07554FF754FF07550FF7551F095
:100C79007552FF81B2E8FAD3E813FC8851C3EF94A7
:100C8900036020EF20E007E82CF8ECFA819EE828C1
:100C99002402F87AFEC3EF940340088A53884D8CE6
:100CA9004F81B288538A4D8C4FE568C33350026433
:100CB9006BF56830600281BC753402D26043E6800E
:100CC900E52D5406602DA840A941C3E913F9E8139D
:100CD900F8306904E92440F9C2AF53E67F75910001
:100CE900C3E498F594E499F595759104D26043E6C7
:100CF90080D2AF22D265754300752000306C037530
:100D09002040020D1CD265754300752040306C03EC
:100D190075200078017901206720E52D54066002CD
:100D2900C2657914E541C313700104F8C3941440F2
:100D3900027814306904781B791BC3E833F8C3E9D6
:100D490033F9206010E543600C306903D53404D2CF
:100D59006DA1D391C40543E59B5440B52002A1BDC3
:100D690030690908C3E899400118A14B20650A08B0
:100D7900C3E8994002A11CA14BC265C2AF53E67FEB
:100D89007591003067127594007595FC759104D2C0
:100D99006043E680D2AFA11CAE40AF41C3EE33FE43
:100DA900EF33FF50047EFF7FFFC3E49EF594E49F79
:100DB900F595A195C3E53394015002A11C30650254
:100DC900A11CD802A1D1A14BC26DC2AF53E67F7558
:100DD9009100855394855495759104854D92854E5E
:100DE90093D26043E680D2AFE52D54066008206AAD
:100DF900020533020E0F306D0D206C0A20650715B0
:100E090081158102169722780030640530650278D1
:100E190001E53775F007A4F9E5F028F5F0E9A2F046
:100E290013A2F113A2F213F537C39478500375375F
:100E390078C3E53795384008D266C295C294C29303
:100E4900306002C149854F92855093D26043E68054
:100E590022207D16C2AF754202D291C2923062023F
:100E6900D293D2AF759F11021051C2AF754202D20F
:100E790091C290306202D295D2AF759F1102105182
:100E8900307245207D22C2AF754203900166757BA1
:100E990002C293D290D292306204D294C1A9C29173
:100EA900D2AF759F01021051C2AF7542039001661E
:100EB900757B02C295D292306204D294C1C9C291A3
:100EC900D2AF759F21021051207D17C2AF75420321
:100ED900900141C293306202D294D2AF759F010250
:100EE9001051C2AF754203900141C295306202D2DE
:100EF90094D2AF759F21021051207D16C2AF754261
:100F090004D292C290306202D294D2AF759F21026C
:100F19001051C2AF754204D290D292C2923062028D
:100F2900D294D2AF759F01021051307243207D20B7
:100F3900C2AF754205900155757B04C294D29130B8
:100F49006204D295E151C292D2AF759F110210513C
:100F5900C2AF754205900177757B01C294D2913079
:100F69006204D293E171C290D2AF759F1102105100
:100F7900207D17C2AF754205900137C294306202D5
:100F8900D295D2AF759F11021051C2AF754205902B
:100F9900014BC2943062EBD293D2AF759F1102100C
:100FA90051207D18C2AF754206D290D292C29130BB
:100FB9006202D295D2AF759F01021051C2AF75423C
:100FC90006D292C291306202D293D2AF759F2102AA
:100FD9001051307245207D20C2AF754201900177D2
:100FE900757B01C295D292306204D293E1F9C29025
:100FF900D2AF759F21021051C2AF754201900155C0
:10100900757B04C293D290D292306204D295011BAF
:10101900C292D2AF759F01021051207D17C2AF75E0
:10102900420190014BC295306202D293D2AF759FB3
:1010390021021051C2AF754201900137C29330624B
:1010490002D295D2AF759F01C26622900135757B98
:1010590000C295C294C293D292D291D290C2622216
:0E106900788076070876070876010876040876
:1010770076FF0876FF08760A087602087601087672
:1010870001788C76010876000876B40876FF087632
:10109700FF0876FF0876030876FF0876010876FFD3
:1010A7000876250876D00876780876C80876040882
:1010B70076FF08760108760008767A08760A0876B9
:1010C700010876010876000876FF087600227887FF
:1010D700E6FFC272BF0302D2727888C27DE630E1B2
:1010E70002D27DC27E7889E630E102D27EC3EF94D8
:1010F700026008758E01D273021107758E00C273E4
:10110700227880E6149000809378A5F67881E6141B
:101117009000809378A6F67886E61490008D9378F1
:10112700A7F6789FE6F8700108C3E89411400278A3
:1011370011E82828F56B256B256B28F56C256B289E
:1011470028F56D7886E6F539C394025003753902A0
:10115700789CE67538FFB402037538A0B4030375AD
:10116700388278A3E61490009A93F56611542222E8
:101177007896E6FA7897E6FB7888E6B40305C3EB3A
:10118700940EFB307F047A007BFFC3EB9AFCC39479
:101197008250027C827572000572EC8572F0A4C3DE
:1011A700E5F0947D40F222D27F31771205B17A00C3
:1011B7007B007C101205A7E55C2AFA74003BFBDC78
:1011C700F37C04C3EB13FBEA13FADCF7FEC27F31AF
:1011D7007722E5EF20E6037520000520903FFFE525
:1011E70020146006901FFF1460009304600375EFDE
:1011F7001253D9BF7581C043FF801205A275EF0254
:1012070043B203E5B3240220E70DF521E5E320E02F
:10121700068521B343E30111547580FF75A400755A
:10122700F19075D47F75908775A5BF75F2BF75D599
:101237000075A60175E2411154E4F8F6D8FD75680A
:101247000111691216F578988673753001C2AF12CD
:1012570005BB1205CB1205B11205D21205B1120555
:10126700D91205B11218171205BB1205BB1205B624
:10127700C2AF78FA79FA308707D9FBD8F7021C0092
:1012870011D531083176317778988673115475A95D
:101297000075B680757A0075881075890275C8243F
:1012A70075910475D84075A82275B80275E69075D2
:1012B7009B80759D0075D10E75BC5875BB0675BAB8
:1012C7001175E8801205A2D2AF12090C75360053CA
:1012D700DACF207E0343DA20307E0343DA1043DA85
:1012E70001C2D8C2711205BBD2617B037A0CE55BE0
:1012F70070077A0CDB030212771205B12070030224
:101307001277C270E55CC3940240E1E52F541F8554
:101317005E5DF55EB55DD5DAD5C26153DACF207E65
:101327000343DA20307E0343DA10C2D8C27178A2B1
:10133700E67008D274E52F54E0F52FC275752900C1
:101347001205B6307409C3E529940A4002D2751212
:1013570005A778023074027800C3E55C9840F0C2B4
:10136700AF1205CB1205CB1205CBD2AF1205BB7559
:101377004C001205A7788CE6C39401500302144F62
:10138700E530C39401500302144F207435C3E55C64
:1013970094FF500302144FC2AF1205E0D2AF1205FB
:1013A700B6C3E55C940150EFC2AF1205CB1205AC92
:1013B7001205CBD2AF1205B6C3E55C94FF40E90234
:1013C700189C7F05D27F31771205B6C2AFC27F3135
:1013D70077AE5CC3E55C947FD2AF40761205A2C2BC
:1013E700AF1205E0D2AFDFDC31AEC3EE94057897DC
:1013F700F61205BB12173612181F7F0AD27F3177F4
:101407001205B6C2AFC27F3177AE5CC3E55C947F8D
:10141700D2AF50E61205A2C2AF1205CB1205AC122D
:1014270005CBD2AFDFD631AEEE24037896F61205A0
:10143700BB12173612184E1205B63177C3E55C9406
:10144700FF5002619102189CC3E55C954C400385EF
:101457005C4C1205B678017988E7B403027805C3B6
:0F146700E55C9840026179C2AF1205E01205E022
:101476001205E0D2AF1205BB753000E4F531F53246
:101486000531E531F4703E0532789AE67819146034
:1014960012783214600D787D14600878FA146003AF
:1014A600753200C3E53298401C11541205A215325C
:1014B60075310078998673C2AF1205E0D2AF78987D
:1014C60086731205B61205ACE52A70053074024122
:1014D6007778012074027806C3E55C9840A212056D
:1014E600B6E52A7003021277C2AF1154E4F522F56D
:1014F60023F524F525F526F567D2AF7885E6C333BF
:10150600F565E4F544F545F546F547F548F570F516
:101516002CF52DF53775700875BB101205A212094A
:101526009FE5E820ECFBA8BDA9BEE97001F888712B
:101536001209A375700875BB1011D5C2AF7561FF8E
:10154600120A5E852261852262852263D2AF7522E8
:1015560001752401752501752601856069756A0185
:1015660075B69075A903757A017888E6B40307C243
:101576007D307602D27DD268D269753300120FAA09
:10158600120FDB120A7E120A85120A7E120A8512D1
:101596000A7E120D0E1206BB120E10120E5A120AF7
:1015A60085120CFD306E0312075B2067031208AF2D
:1015B6003067031208F6120E10120E89120A8512EF
:1015C6000D0E306E03120797120E10120F02120A3A
:1015D60085120CFD306E031207F5120E10120F3332
:1015E600120A85120D0E306E03120853120E1012D7
:1015F6000FAA120A8512099F120CFD120E10120F65
:10160600DB1209A3120A8530692C85646185646240
:10161600856069756A0179187A0CC3E533994009C2
:10162600C269D26A8A3502163CC3E55C940140035E
:1016360002159802169F306A1D206C1AE535147043
:1016460006C26AD26BA198F535C3E55C94014003E6
:1016560002159802169F753600C3E55F940140098E
:10166600856462856069756A0178FA79A4E7600223
:101676007803C3E55F985021307404E52A601A7830
:10168600F0306C058564617820C3E541985002A16D
:10169600980536E55C6002C1A2753600C2AF1154EA
:1016A6007887E6FE760211D57887EEF6E4F522F520
:1016B60023F524F525F526F565752C00752D0075A1
:1016C600A90075B680757A00D2AF1205B6115478A6
:1016D600A4E66006C292C291C290307406E52A70F2
:1016E600024177788DE6C39401400261568181906C
:1016F6001A0D7820121778E520B4A50CA3121778D6
:10170600E520B45A03021716116912173602173567
:10171600901A0378807B0A121778A308DBF9901ACF
:101726000F788C7B19121778A308DBF9901A2822F8
:10173600C2AF1217B7121791901A00740E12177DC6
:10174600A3740612177DA3741512177D901A0378D9
:10175600807B0A12177CA308DBF9901A0F788C7B22
:101766001912177CA308DBF91217CA1217A8901AC8
:101776002822E493F622E6438F01538FFD75EF028C
:1017860075B7A575B7F1F0538FFE22438F02438FCD
:101796000175EF0275B7A575B7F1901A0DF0538F65
:1017A600FC22901A0D74A5F17D901A0E745AF17DE3
:1017B600227A3079D07820901A40F178E520F7091E
:1017C600A3DAF7227A3079D0901A40E7F17D09A39F
:1017D600DAF922AB74A875BB01027980BB020279E3
:1017E60081BB03027982BB04027994BB050279832B
:1017F600BB06027986BB07027992BB08027987BBD2
:101806000902799CBB0A027988BB0B027989E8F741
:10181600227C051205BBDCFB22C2AF1205CB1205EA
:10182600D21205D91205E01205AC1205CB1205D26B
:101836001205D91205E01205AC1205CB1205D2121B
:1018460005D91205E0D2AF22C2AF1205E01205D9C2
:101856001205D21205CB1205AC1205E01205D912FB
:0E18660005D21205CB1205AC1205E01205D911
:101874001205D21205CBD2AF22AE74AF75C2AF122D
:1018840005CB1205CB1205CB1205ACDEF21205E036
:101894001205ACDFF8D2AF22111F1117111775749E
:1018A40001757501757600117D7C05AD5C1205BB73
:1018B400C3ED955C70F5C3E55C9401400AC3E55C37
:1018C40094FF40340218DA1217D9121736111FC2C6
:1018D400AF75EF121117DCD30576C3E57694035088
:1018E4000280C411170575E5741490009F93F808DD
:1018F400C3E57598500280AC111711170574C3E540
:1019040074940C5002809A121069121736C2AF7583
:04191400EF121117A6
:0319FD000211D9FB
:101A00000E061507070104FFFF0A020101A55A018E
:101A100000B4FFFFFF03FF01FF25D078C804FF01DA
:091A200000FF0A010100FF00FFB4
:101A4000234F76736B794D5232304150726F2320A1
:101A500023424C48454C492346333930232020202B
:101A60002020202020202020202020202020202076
:101C0000C2AFC2D353D9BF7581C043B20343FF8073
:101C1000752438752503B1C975EF0275E24043F1AB
:101C20008053A47F75D4FFD2877DFA780379E67C50
:101C300010752200752300901DD67B0675249875BB
:101C400025013087028142208708D8FBD9F9DCF7CB
:101C500081B4308708D8FBD9F9DCF781B4B189E4C5
:101C600093A3C39A6004DDC381B4DBDBB17B600264
:101C7000812B7B08E493FAA3B15CDBF87A30B15C8A
:101C8000752200752300B17BEAFCEBFDC3ED94FEE9
:101C9000400EB17B8A278B28ED30E0048A828B834B
:101CA000B17B7AC270D8C3ED94FE601350CEBD00F4
:101CB00025EC60097520007521FF0200008100A855
:101CC00027A9280809D804D90281D3B17FEA89AAB3
:101CD000F281C50D81A0C3ED94035049EDA2E092BD
:101CE000007AC5C3E5829400E583941C50902000DF
:101CF00010438F02438F0175B7A575B7F1F030001F
:101D00001FA827A9280809438F01538FFDD804D99C
:101D100002A12089AAE275B7A575B7F1F0A3A10DBC
:101D2000538FFC817C7AC1BD030CE493A3FAB140CC
:101D3000DCF8B138817C817EAA22AB23B15CEBFA5E
:101D4000EA6222752608C3E52313F523E52213F57D
:101D50002250066323A0632201D526EAB1C9B1C986
:101D600075260AEAF4200102D287300102C287B147
:101D7000C9C3134002C201D526EB22B17FEAFB2082
:101D80008702A17F308702A184752608AE24AF2583
:101D9000C3EF13FFEE13FEB1CDB1C9C3EA13308711
:101DA000024480FA30E703632201C3E52313F523DD
:101DB000E52213F52250066323A0632201D526D91C
:101DC000E52265236523F52222AE24AF250E0FDE22
:101DD000FEDFFCD20122424C48656C693437316326
:041DE000F390060175
:00000001FF
